:100000000C945C000C9447050C9474050C948400CB
:100010000C9484000C9484000C9484000C94840050
:100020000C9484000C9484000C9484000C94840040
:100030000C9484000C9484000C9484000C94840030
:100040000C94A1050C9484000C9403070C94840078
:100050000C9484000C9484000C9484000C94840010
:100060000C9484000C948400000024272A000025AE
:10007000282B000023262904040404040404040299
:100080000202020202030303030303010204081035
:100090002040800102040810200102040810200002
:1000A0000000070002010000030406000000000039
:1000B0000000000058022D0411241FBECFEFD4E031
:1000C000DEBFCDBF11E0A0E0B1E0ECE6F2E102C09E
:1000D00005900D92A031B107D9F712E0A0E1B1E08F
:1000E00001C01D92A432B107E1F710E0C8EBD0E0E7
:1000F00004C02297FE010E943009C43BD107C9F712
:100100000E9426040C9434090C940000FC014487DE
:100110005587668777870895CF93DF93EC01EC8D41
:10012000FD8D9081888D809589238083E8A1F9A138
:1001300090818E8D809589238083ECA1FDA1908193
:100140008E8D809589238083E8A1F9A180819E8D81
:10015000892B8083E8A1F9A190818E8D80958923D8
:100160008083EC8DFD8D8081988D892B8083EAA121
:10017000FBA180816E8D90E0262F30E082239323B7
:10018000892BB1F42C893D894E895F8988859985B1
:10019000AA85BB85281739074A075B0748F42F5FF4
:1001A0003F4F4F4F5F4F2C8B3D8B4E8B5F8BDFCF85
:1001B0002C893D894E895F8988859985AA85BB856B
:1001C00082179307A407B50708F440C0ECA1FDA16E
:1001D0008081682B6083E8A1F9A180819E8D892BA5
:1001E0008083E8A1F9A190818E8D809589238083F9
:1001F000ECA1FDA190818E8D809589238083EC8D6B
:10020000FD8D9081888D809589238083EAA1FBA153
:10021000208130E08E8D90E028233923232BE1F0DC
:100220002C893D894E895F8988859985AA85BB85FA
:10023000281739074A075B0778F42F5F3F4F4F4F66
:100240005F4F2C8B3D8B4E8B5F8BE0CF2EEF3FEFC4
:10025000C901DF91CF9108952C893D894E895F892D
:1002600088859985AA85BB85281739074A075B07C2
:1002700068F721E030E0ECCFEF92FF920F931F93ED
:10028000CF93DF93EC01062F1C8A1D8A1E8A1F8ADA
:10029000662329F420E030E040E050E07FC0888110
:1002A000998197FF05C02FEF3FEF4FEF5FEF76C0CB
:1002B00010E0CE010E948C0097FF05C02EEF3FEFAB
:1002C0004FEF5FEF6BC01F5F101798F30E9411068E
:1002D000288939894A895B89621B730B840B950BCA
:1002E0002C853D854E855F852617370748075907BA
:1002F000C0F52C893D894E895F896A817B818C811B
:100300009D81261737074807590721F4EE24FF245B
:10031000870106C079018A01E61AF70A080B190B52
:100320000E94BA072DEC3CEC4CEC5DE30E944808BF
:100330000E948907882777FD8095982FE616F70693
:100340000807190770F48FEF9FEFAFEFBFE08A83C4
:100350009B83AC83BD830E941106688B798B8A8B4B
:100360009B8B2C893D894E895F898A819B81AC81D9
:10037000BD81281739074A075B0720F42A833B838E
:100380004C835D832C893D894E895F898A819B815D
:10039000AC81BD81281B390B4A0B5B0BB901CA012B
:1003A000DF91CF911F910F91FF90EF900895CF9320
:1003B000DF93EC0181E090E09983888386E391E00C
:1003C0009F838E8380EF9AEBA4E0B0E088879987C3
:1003D000AA87BB8780E29EE4A0E0B0E08C879D877F
:1003E000AE87BF87862F90E0FC01E557FF4FE49171
:1003F000E88F89589F4FFC016491698FE62FF0E0E8
:10040000E359FF4FE491EC8F1D8E842F90E0FC01A7
:10041000E557FF4FE491EE8F89589F4FFC014491BF
:100420004F8FE42FF0E0E359FF4FE491ECA31DA2BE
:10043000662321F48FEF9FEF99838883E98DF0E0A5
:10044000E859FF4FE491EA8F1B8E8F8D882321F4AA
:100450008FEF9FEF99838883EF8D8E2F90E0FC01C3
:10046000E859FF4FE491E8A319A2FC01E359FF4FBB
:10047000E491ECA31DA28E589F4FFC0184918AA3A6
:100480001BA2EA8DFB8D8081988D892B80838FEF55
:100490009FEFAFEFBFE08A839B83AC83BD830E9455
:1004A0001106688B798B8A8B9B8BDF91CF91089596
:1004B00042E064E080E191E00E94D70145E064E021
:1004C00086E391E00E94D70148E064E08CE591E08A
:1004D0000E94D70108952F923F924F925F926F92A0
:1004E0007F928F929F92AF92BF92CF92DF92EF92C4
:1004F000FF920F931F93DF93CF93CDB7DEB728976B
:100500000FB6F894DEBF0FBECDBF0E9411066D83FB
:100510007E838F8398876EE180E191E00E943C01A9
:100520003B014C016EE186E391E00E943C011B011E
:100530002C016EE18CE591E00E943C0169837A8395
:100540008B839C83E0908801F09089010027F7FC61
:100550000095102F2091040130910501442737FDAB
:100560004095542F8FEF90E0A0E0B0E0BF93AF93A1
:100570009F938F93AA24BB246501C401B3010E94F9
:1005800040070F900F900F900F906F3F710519F07B
:1005900014F06FEF70E077FF02C060E070E07093DE
:1005A000830160938201E0908A01F0908B01002723
:1005B000F7FC0095102F2091060130910701442788
:1005C00037FD4095542F8FEF90E0A0E0B0E0BF934F
:1005D000AF939F938F93AA24BB246501C201B101FD
:1005E0000E9440070F900F900F900F906F3F710582
:1005F00019F014F06FEF70E077FF02C060E070E078
:100600007093850160938401E0908C01F0908D01DE
:100610000027F7FC0095102F209108013091090167
:10062000442737FD4095542F8FEF90E0A0E0B0E0D5
:10063000BF93AF939F938F93AA24BB2465016981D5
:100640007A818B819C810E9440070F900F900F90C0
:100650000F906F3F710519F014F06FEF70E077FFA6
:1006600002C060E070E070938701609386010E9491
:100670001106AB01BC018D819E81AF81B885481BFD
:10068000590B6A0B7B0B8EE891E00E94040560E039
:1006900071E08EE891E00E943D04609182017091CA
:1006A00083018EE891E00E942F0560E071E08EE802
:1006B00091E00E943D0460918401709185018EE873
:1006C00091E00E942F0560E071E08EE891E00E94C9
:1006D0003D0460918601709187018EE891E00E944F
:1006E000370528960FB6F894DEBF0FBECDBFCF9169
:1006F000DF911F910F91FF90EF90DF90CF90BF900F
:10070000AF909F908F907F906F905F904F903F90B1
:100710002F90089561E08DE00E94590661E08DE020
:100720000E9477064FEF5FEF6FEF7FEF80E191E080
:100730000E9486004FEF5FEF6FEF7FEF86E391E05F
:100740000E9486004FEF5FEF6FEF7FEF8CE591E047
:100750000E94860066C06EE180E191E00E943C014B
:1007600070938301609382016EE186E391E00E94C1
:100770003C0170938501609384016EE18CE591E00A
:100780000E943C01AB017093870160938601209128
:1007900082013091830180918801909189018217B3
:1007A000930724F4309389012093880180910401F8
:1007B000909105012817390724F4309305012093FF
:1007C0000401209184013091850180918A019091EA
:1007D0008B018217930724F430938B0120938A01B5
:1007E00080910601909107012817390724F430936E
:1007F00007012093060180918C0190918D0184174F
:10080000950724F450938D0140938C018091080149
:10081000909109014817590724F450930901409316
:1008200008010E941106605177428040904008F410
:1008300092CF60E08DE00E94770640E05BE460E0EC
:1008400070E08EE891E00E94380408950E941F062F
:100850000E948A030E946B02FDCF8EE091E090938C
:100860008F0180938E010895862F0E94FB060895C4
:10087000CB01BA010E94C20608950F931F93CF9334
:10088000DF938C01EB0109C02196D801ED91FC9119
:100890000190F081E02DC801099568816623A1F7D8
:1008A000DF91CF911F910F9108950F931F938C01AA
:1008B000DC01ED91FC910190F081E02D6DE0099556
:1008C000D801ED91FC910190F081E02D6AE0C80122
:1008D00009951F910F9108952F923F924F925F9229
:1008E0006F927F928F929F92AF92BF92CF92DF9240
:1008F000EF92FF920F931F93DF93CF93CDB7DEB7A5
:10090000A0970FB6F894DEBF0FBECDBF1C016A01E1
:100910007B01411551056105710549F4DC01ED913B
:10092000FC910190F081E02D60E3099554C088248A
:1009300099245401422E55246624772401E010E0C6
:100940000C0F1D1F080D191DC701B601A30192014F
:100950000E94DD08F80160830894811C911CA11C91
:10096000B11CC701B601A30192010E94DD08C901B3
:10097000DA016C017D01C114D104E104F104F1F646
:1009800081E0E82EF12CEC0EFD1EE80CF91C3E0176
:100990000894611C711CD501C4010197A109B1091A
:1009A0006C01C818D90814C0F601EE0DFF1D608156
:1009B0006A3010F4605D01C0695CD101ED91FC9179
:1009C0000190F081E02DC10109950894E108F1083A
:1009D0006E147F0449F7A0960FB6F894DEBF0FBEE1
:1009E000CDBFCF91DF911F910F91FF90EF90DF90DE
:1009F000CF90BF90AF909F908F907F906F905F90BF
:100A00004F903F902F9008952AE00E946C04089523
:100A1000EF92FF920F931F93CF93DF93EC017A0134
:100A20008B0177FF0FC0E881F9810190F081E02D03
:100A30006DE2099510950095F094E094E11CF11C8D
:100A4000011D111D2AE0B801A701CE010E946C040E
:100A5000DF91CF911F910F91FF90EF900895AB011F
:100A6000662757FD6095762F0E94080508950F931D
:100A70001F938C01AB01662757FD6095762F0E946E
:100A80000805C8010E9455041F910F9108951F92F7
:100A90000F920FB60F9211242F933F934F935F93B2
:100AA0006F937F938F939F93AF93BF93EF93FF9336
:100AB0008091900190919101892B29F0E091900112
:100AC000F09191010995FF91EF91BF91AF919F91A5
:100AD0008F917F916F915F914F913F912F910F90E7
:100AE0000FBE0F901F9018951F920F920FB60F9286
:100AF00011242F933F934F935F936F937F938F9323
:100B00009F93AF93BF93EF93FF9380919201909146
:100B10009301892B29F0E0919201F09193010995BD
:100B2000FF91EF91BF91AF919F918F917F916F91C5
:100B30005F914F913F912F910F900FBE0F901F909B
:100B400018951F920F920FB60F9211242F938F9327
:100B50009F93AF93BF938091940190919501A09141
:100B60009601B09197010196A11DB11D809394014A
:100B700090939501A0939601B0939701809198016D
:100B800090919901A0919A01B0919B018050904C55
:100B9000AF4FBF4F8093980190939901A0939A0112
:100BA000B0939B0127C08091980190919901A091E9
:100BB0009A01B0919B0180549F41A040B040809326
:100BC000980190939901A0939A01B0939B01809111
:100BD0009C0190919D01A0919E01B0919F01019671
:100BE000A11DB11D80939C0190939D01A0939E0136
:100BF000B0939F018091980190919901A0919A01E1
:100C0000B0919B0181549F41A040B04060F6BF91DC
:100C1000AF919F918F912F910F900FBE0F901F90CA
:100C200018958FB7F89420919C0130919D014091C7
:100C30009E0150919F018FBFB901CA010895789418
:100C400084B5826084BD84B5816084BD85B58260D1
:100C500085BD85B5816085BDEEE6F0E0808181606F
:100C60008083E1E8F0E08081826080838081816020
:100C70008083E0E8F0E0808181608083E1EBF0E058
:100C8000808184608083E0EBF0E0808181608083FC
:100C9000EAE7F0E0808184608083808182608083E5
:100CA0008081816080838081806880831092C10010
:100CB0000895282F30E0C90185579F4FFC0194917A
:100CC00029583F4FF9018491882381F0E82FF0E003
:100CD000E859FF4FE491F0E0662329F48081909574
:100CE0008923808308958081892B80830895482FEC
:100CF00050E0CA0181569F4FFC012491CA018557DB
:100D00009F4FFC01949149585F4FFA01349133236E
:100D1000C1F1222331F1233021F4809180008F77BB
:100D200005C0243031F4809180008F7D8093800055
:100D300018C0213019F484B58F7704C0223021F413
:100D400084B58F7D84BD0DC0263021F48091B00024
:100D50008F7705C0273029F48091B0008F7D809374
:100D6000B000E32FF0E0E359FF4FE491F0E0662399
:100D700029F4808190958923808308958081892B2F
:100D800080830895EF92FF920F931F937B018C0154
:100D900022E030E040E050E00E94FF08205E3E4547
:100DA000484F5F4FCA01B901A80197010E94FF088F
:100DB000C901DA010197A109B109292F3A2F4B2F57
:100DC000552747FD5A950196A11DB11D2093C500D9
:100DD00081508093C400E1ECF0E0808180618083E9
:100DE0008081886080838081806880831F910F91DB
:100DF000FF90EF900895982F8091C00085FFFCCF61
:100E00009093C60008951F920F920FB60F9211246F
:100E10002F933F934F935F936F937F938F939F9302
:100E2000AF93BF93EF93FF934091C600E091A00171
:100E3000F091A101CF01019660E870E00E94CA081C
:100E40009C018091A2019091A3012817390739F0E4
:100E5000EC55FE4F40833093A1012093A001FF91F8
:100E6000EF91BF91AF919F918F917F916F915F9122
:100E70004F913F912F910F900FBE0F901F9018959B
:100E80002F923F924F925F926F927F928F929F929A
:100E9000AF92BF92CF92DF92EF92FF920F931F9388
:100EA000DF93CF93CDB7DEB73B014C0119012A0187
:100EB0006D897E898F89988D6A197B098C099D09B6
:100EC000621A730A840A950AA40193010E94AB086E
:100ED000E218F30804091509A80197010E94FF0808
:100EE0002A0D3B1D4C1D5D1DB901CA01CF91DF913B
:100EF0001F910F91FF90EF90DF90CF90BF90AF9038
:100F00009F908F907F906F905F904F903F902F9029
:100F1000089504D06894B111B5C0089598D088F0B0
:100F20009F5790F0B92F9927B751A0F0D1F0660FD5
:100F3000771F881F991F1AF0BA95C9F712C0B130F0
:100F400081F09FD0B1E008959CC0672F782F88274B
:100F5000B85F39F0B93FCCF3869577956795B3952F
:100F6000D9F73EF490958095709561957F4F8F4F9E
:100F70009F4F0895E89409C097FB3EF490958095A3
:100F8000709561957F4F8F4F9F4F9923A9F0F92F4F
:100F900096E9BB279395F695879577956795B795CD
:100FA000F111F8CFFAF4BB0F11F460FF1BC06F5FB3
:100FB0007F4F8F4F9F4F16C0882311F096E911C0C5
:100FC000772321F09EE8872F762F05C0662371F0E6
:100FD00096E8862F70E060E02AF09A95660F771FFA
:100FE000881FDAF7880F9695879597F9089597F9EE
:100FF0009F6780E870E060E008959FEF80EC0895BF
:1010000000240A94161617061806090608950024E7
:101010000A9412161306140605060895092E039461
:10102000000C11F4882352F0BB0F40F4BF2B11F4D5
:1010300060FF04C06F5F7F4F8F4F9F4F089557FD34
:101040009058440F551F59F05F3F71F04795880F36
:1010500097FB991F61F09F3F79F0879508951216CD
:1010600013061406551FF2CF4695F1DF08C0161679
:1010700017061806991FF1CF86957105610508942A
:101080000895E894BB2766277727CB0197F9089541
:101090000BD0C4CFB5DF28F0BADF18F0952309F0E4
:1010A000A6CFABCF1124EECFCADFA0F3959FD1F32B
:1010B000950F50E0551F629FF001729FBB27F00D06
:1010C000B11D639FAA27F00DB11DAA1F649F66275B
:1010D000B00DA11D661F829F2227B00DA11D621FAA
:1010E000739FB00DA11D621F839FA00D611D221F64
:1010F000749F3327A00D611D231F849F600D211D48
:10110000822F762F6A2F11249F5750408AF0E1F0EA
:1011100088234AF0EE0FFF1FBB1F661F771F881F33
:1011200091505040A9F79E3F510570F060CFAACF73
:101130005F3FECF3983EDCF3869577956795B7951E
:10114000F795E7959F5FC1F7FE2B880F911D969548
:10115000879597F90895629FD001739FF001829F50
:10116000E00DF11D649FE00DF11D929FF00D839F36
:10117000F00D749FF00D659FF00D9927729FB00DD3
:10118000E11DF91F639FB00DE11DF91FBD01CF01E6
:101190001124089597FB092E07260AD077FD04D065
:1011A00049D006D000201AF4709561957F4F0895BC
:1011B000F6F7909581959F4F0895A1E21A2EAA1BEC
:1011C000BB1BFD010DC0AA1FBB1FEE1FFF1FA217F7
:1011D000B307E407F50720F0A21BB30BE40BF50BF4
:1011E000661F771F881F991F1A9469F7609570957D
:1011F000809590959B01AC01BD01CF01089597FBAF
:10120000092E05260ED057FD04D0D7DF0AD0001CCA
:1012100038F450954095309521953F4F4F4F5F4F93
:101220000895F6F790958095709561957F4F8F4F53
:101230009F4F0895AA1BBB1B51E107C0AA1FBB1FEC
:10124000A617B70710F0A61BB70B881F991F5A9552
:10125000A9F780959095BC01CD010895EE0FFF1F71
:0C1260000590F491E02D0994F894FFCF64
:10126C0020202000FF03FF03FF03000000003404D4
:00000001FF
